:084FEA0041086501C107C10681
:105B010090085AE090084BF090085BE090084AF04A
:105B110090085CE090084DF090085DE090084CF032
:105B210022900866E0FF900859E06F2290085AE041
:105B3100900828F090085BE0900829F090085CE05C
:0D5B410090082AF022F09008657401F0220F
:101A1B0030B60930B7037F2C227F2D2230B7037FDE
:051A2B002E227F2F2296
:101389009006DE7401F0E4A3F0A3F0A3F0A3F075D6
:10139900FFDE75FFADF5E6F5E7125B981262801284
:1013A900630B125409125DB3121A1B900866EFF011
:1013B900D2AF124200125F08EF605A1259BAEF24F5
:1013C900F8601C24F8601D24F0601E24E0602224CB
:1013D900C06036247C70353006261262D4802D1206
:1013E900609080081261B98003125FC112619C800C
:1013F9001B30060C900866E0FF7D11126122800CFB
:10140900E4FF1261D4C20780031248A5125B471298
:101419005F08EF70A690085EE06401600302151A88
:10142900900858E0FFB40B05D206125B47EF643110
:101439007031125B22600302151A126040EF60FAE4
:1014490012163C126040EF60FA125B0112516712EA
:101459006040EF60FA121645126040EF6003021512
:101469001A80F5900858E06432702E125B226003EE
:1014790002151A126040EF60FA12163C126040EF32
:1014890060FA125B01124E47126040EF60FA1216C1
:1014990045126040EF707A80F8900858E0642D702A
:1014A90035125B22706B126040EF60FA900866E0BB
:1014B900FF1262BF126040EF60FA125B2D12537681
:1014C900126040EF60FA900866E0FF1262AA1260AB
:1014D90040EF703D80F8900858E0642E7033125B3D
:1014E90022702E126040EF60FA900866E0FF1262E7
:1014F900BF126040EF60FA125B2D12552512604051
:10150900EF60FA900866E0FF1262AA126040EF608D
:10151900FA90085EE06401704C900867E030E022C0
:10152900900858E020E71B14600D047015900859C5
:10153900E0FF1262228008900859E0FF1261D4127C
:101549005B47900858E0FDB41409900867E044012E
:10155900125B46EDB41509900867E054FE125B462C
:10156900E490085EF0300E1AE49006E2F09006E28C
:10157900E0FFC3940F500B1210899006E2E004F0CB
:1015890080EB900407E0FF7E00C39455EE94005071
:1015990007E49006DEF08014C3EF94AAEE9400905D
:1015A90006DE50057401F080037402F09006DFE056
:1015B900FF9006DEE0FE6F6003125B479006DFEEE8
:1015C900F0900867E0C413135403FFBF022090088A
:1015D90038E0FCA3E0FDD39400EC9480400590062C
:1015E900E08016C3EC9480501A9006E08010EF70EA
:1015F90012E50C9006E030E7057401F0800A74FFEB
:10160900F08005E49006E0F09006E1E0FF9006E046
:10161900E0FE6F6003125B479006E1EEF09008650B
:10162900E0640160030213BB123DC9E4900865F050
:031639000213BBDE
:10163C00900866E0FF1262BF22900866E0FF12621B
:02164C00AA22D0
:104FF200410773004107770043076D00020741072D
:1050020074004107700050074B00000000000000D0
:1050120000000000000000000050075B00000000DC
:0C50220000000000000000000000000082
:105AB30090072CE025E025E0245BF582E4340722FF
:105AC300F58312101A90072DE0FEA3E0FF22FF7C5E
:105AD300007D07120DE8AC06AD0790073BE0FEA37F
:105AE300E078032225E025E0244BF582E434072205
:0E5AF300F583E0F8A3E0F9A3E0FAA3E0FB22BC
:06616200900770E07016CA
:1061680090073EE584F0E4F58490077004F0D2ECE3
:0661780090073EE0F584F3
:01617E0022FE
:1052DC00AF84E4F584900774E0600302537304F028
:1052EC00900773E0FE5403FDEE1313543FFEC2FF10
:1052FC00ED14602714603914605524037069C2A141
:10530C00D2A0D2A3D2A2E59A20E7FB20FFF830F975
:10531C00F5EE33333354F8F59B804CC2A2D2A0D2B5
:10532C00A3D2A1E59A20E7FB20FFF830F9F5801312
:10533C00C2A3D2A0D2A2D2A1E59A20E7FB20FFF80B
:10534C0030F9F5EE33333354F84404F59B8018C22E
:10535C00A0D2A3D2A2D2A1E59A20E7FB20FFF8307D
:09536C00F9F5EE4430F59B8F8445
:015375002215
:031A1500024AA9D9
:104AA900C0E0C0F0C083C082C0D075D000C000C0D3
:0D4AB90001C002C003C004C005C006C00754
:104AC600A2AF9202900773E0FF5403FEEF13135454
:104AD6003F900723F0EE7003FF80027F01900724CA
:104AE600EFF0900722E584F0758400C2FFEEC394D0
:104AF60003505E900726E59BF0E59A20E7FB20FF32
:104B0600F830F9F5759B0030FFFDC2FF900727E5E9
:104B16009BF0EE541F33333354F8FF900725E054CF
:104B2600074FF0900723E0145407FF900725E05441
:104B3600F84FF0900727E0C4F8540FC868FD9007B7
:104B460026E0C454F048FC900725E0FF12187F8049
:104B560008900723E0FF124D73D2A0D2A3D2A2D2AF
:104B6600A1900773E004F0D3941F4002E4F090078D
:0F4B760074E4F0C2FFA20292AF900722E0F58430
:104B8500D007D006D005D004D003D002D001D00084
:0B4B9500D0D0D082D083D0F0D0E0322E
:031A30000252243B
:10522400C0E0C0F0C083C082C0D075D000C000C050
:0752340004C005C006C0071D
:10523B0090073BE5BFF0A3E5BEF0900777E0146065
:10524B00271460442402704F90076B125AE0CEC3B0
:10525B0013CE13D8F9125AD1CEC313CE13D8F92DBE
:10526B00FFEC3E90076B802B900771125AE0CEC378
:10527B0013CE13D8F9125AD1CEC313CE13D8F92D9E
:10528B00FFEC3E900771800B90073BE0FFA3E09093
:10529B000775CFF0A3EFF0900777E004F0E0C3942D
:1052AB00034002E4F0900777E0246DF582E43407C5
:0C52BB00F583E0F5BB900770E4F0C2ED55
:1052C700D007D006D005D004D000D0D0D082D0836C
:0552D700D0F0D0E03230
:0C50AA0090072CEFF0F9A3ECF0A3EDF060
:1050B600FFAE04E4FCFDE9125AE7125AF3C3120FDD
:1050C600AE5027125AC8E4FCFD90072CE0FB125A9A
:1050D600E7125AC3EF24F8FFEE34FFFEE434FFFD77
:1050E600E434FFFCEB125AB78034125AC8E4FCFDD4
:1050F600125AB3125AF3D3120FAE4027125AC8E40B
:10510600FCFD90072CE0FB125AB7125AC3EF240895
:10511600FFE43EFEE433FDE433FCEB125AE7F5838D
:1051260012101A125AB3F583E0FCA3E0FDA3E0FEC9
:10513600A3E0FFE47BFF7AFFF9F8C3120FAE500A33
:1051460074FF90072DF0A3F08013125AB3F583A3D2
:10515600A3E0FFA3E090072DCFF0A3EFF0125AC80B
:015166002226
:1049A90050505050505050505050505051515151FA
:1049B90051515151515152525252525252525253D3
:1049C90053535353535353545454545454545555A3
:1049D900555555555656565656565757575757576C
:1049E900585858585859595959595A5A5A5A5B5B2B
:1049F9005B5B5B5C5C5C5C5D5D5D5E5E5E5E5F5FE0
:104A09005F5F606060616161626262636363646485
:104A190064656565666667676768686969696A6A1A
:104A29006B6B6C6C6D6D6E6E6E6F6F707171727297
:104A39007373747475757677777879797A7A7B7CFC
:104A49007C7D7E7F7F80818182838485858687883E
:104A590089898A8B8C8D8E8F909192939495969754
:104A690098999A9B9C9D9E9FA0A2A3A4A5A6A8A93C
:104A7900AAABADAEAFB1B2B4B5B7B8B9BBBCBEC0E5
:104A8900C1C3C4C6C8C9CBCDCFD0D2D4D6D8DADC3D
:104A9900DEE0E2E4E6E8EAECEEF1F3F5F7FAFCFF32
:10502E0042084E0000420850000042085200004262
:0A503E000854000041085601C10C9F
:1056AB00E0C4F854F0C868FEA3E0C4540F48FFEE02
:1056BB00540FFEEF25E0FFEE33FE74362FF58274A8
:1056CB001A3EF583E493FE74019322E0FFA3E0CF2F
:1056DB00900728F0A3EF2224ABFFEF7F00FE7C00A6
:1056EB007D55020DFA74A92BF58274493AF583E4C2
:1056FB00937F00FE22900407E0FF7E00C39455EEDB
:10570B00940022E0FFA3E0A3CFF0A3EFF0229008D8
:08571B0067E013131354072289
:0A633B00AF84E4F58475D4948F84D8
:016345002235
:0A634600AF8475840175D4948F8430
:01635000222A
:105E2B001257005002801AC3EF94AAEE9400EF5061
:105E3B000D1256E2C374FF9FFBE49EFA800A2456B0
:105E4B00FF1256E5AA06AB07D3EB94FFEA9400408A
:085E5B00047A007BFF1256F0EF
:015E6300221C
:105E640012570050028016C3EF94AAEE9400EF502C
:105E7400091256E2AA06AB07800E2456FF1256E515
:105E8400C374FF9FFBE49EFAD3EB94FFEA940040B3
:075E940003E4FAFB1256F0D3
:015E9B0022E4
:104D7300A984E4F584A2AF9203EFB40800400302D0
:104D83004E15904D8CF8282873024DA4024DD10284
:104D93004DDB024DE5024DEF024DAC024DF9024EE3
:104DA3000412571930E21E800612571930E116C259
:104DB300AF900406E025E0FE900405E03390072859
:104DC300F0A3CE8048E4900728F0A3F08044C2AF5C
:104DD3009004071256D68035C2AF9006351256D6C8
:104DE300802BC2AF9006331256D68021C2AF9006F5
:104DF300311256D68017C2AF125E2BEE1256DB80ED
:104E03000CC2AF125E64900728EEF0A3EFF0A2038A
:104E130092AF900728E0F59B30FFFDC2FFE59A2093
:104E2300E7FB20FFF830F9F5900729E0F59B30FF09
:104E3300FDC2FFD2A0D2A3D2A2D2A1A20392AFAF4E
:034E4300018F8458
:014E46002249
:031A3300023F4C23
:103F4C00C0E0C0F0C083C082C0D075D000C000C03B
:0D3F5C0001C002C003C004C005C006C007BC
:103F690090073DE584F0C2CF758403124F1A300DD6
:103F790017C3920D900867E0135403FFBF0109901E
:103F89000852E4F0A3F0806E900867E0F9C3135477
:103F990003FF6402703B900852E0FCA3E0FDC3EC10
:103FA90094E04002D20C300C4D90084EE0A320E77B
:103FB90045A3E0A330E73FD3ED94FFEC941F4006FF
:103FC900A3E094E04030900852E4F0A3F0C20C80E2
:103FD90025EF64037020900852E020E7047F0180F8
:103FE900027F0090084EE020E7047E0180027E00F7
:103FF900EE6F24FF92909008521256ABFDAC0678F2
:1040090005C333CE33CED8F9FDAC068C0CF50DECD7
:104019006480FC90084E1256ABFBAA067805C333A0
:10402900CE33CED8F9FBAA06EA6480FA758400ED8E
:10403900F5D2ECFF8FD3758401AF03EFF5D2AE0251
:10404900EEFF8FD390084E12570E90084FE02511BE
:10405900F090084EE03510F090085212570EA3E088
:1040690014F07024900853E0250FF0900852E035C1
:104079000EF0900867E0C41313540370047F0480A2
:10408900027F01900856EFF01261621252DC90072C
:044099003DE0F5848D
:10409D00D007D006D005D004D003D002D001D00077
:0B40AD00D0D0D082D083D0F0D0E03221
:105FEC00781AE0FEA3E0A60608F622781CE0FEA3D1
:105FFC00E0A60608F622E6FE08E6F5828E832292DB
:0A600C00AFAF028FB1AF038F842203
:10596200AB84AAB1A2AF920190071212101A90074B
:1059720014125FEC53B10F900713E0700543B1109E
:105982008019900714E030E70543B130800D43B130
:1059920020900714E04480F0125FECE4F584C2AF7B
:1059A20043B701758F03781A126002E4F053B7FE11
:0759B200F58FA20112600B4A
:0159B90022CB
:10572300AB84AAB1A2AF920190071E12101A900780
:105733001DE0F9FF3395E0FEEFF44E60499007203A
:10574300781A125FEE53B10F90071FE0700543B153
:1057530010801B900720E030E70543B130800F43F2
:10576300B120900720E04480F0781A125FF9E4F545
:1057730084C2AF43B701758F01781A126002E9F052
:0B57830053B7FEE4F58FA20112600B8B
:01578E0022F8
:0F58B00090072CEBF0A3EAF0A3E9F0A312101A73
:1058BF00E4900735F0A3F0900733E0FEA3E0FFC3B9
:1058CF00900736E09F900735E09E502D90072F12DE
:1058DF000FE5125BE190072CE0FBA3E475F00112DA
:1058EF000E65A9F0FAEF120DD6900736E004F070AE
:0958FF00C6900735E004F080BEFC
:01590800227C
:105BE100AB84AAB190073712101A900739125FF7E8
:105BF10053B10F900738E0700543B1108019900739
:105C010039E030E70543B130800D43B120900739C9
:105C1100E04480F0125FF7781C126002E493FFAE5B
:075C2100028EB1AE038E8478
:015C28002259
:1050480001150001120002180000011700011600E6
:0C505800021300004107A9004107AF004F
:106101009007ACE0FBA3E0FAA3E0F92204F0A3744A
:1061110007F0A374B3F022FF9007AAEAF0A3EFF00F
:01612100225B
:055630009006E3EFF01D
:105635009007AAE0FEA3E0FF2401FDE43EFAA905D8
:105645009006E47401F0A3EAF0A3E9F09006E412F1
:10565500610474019007F36B7008E965827003EAD1
:10566500658370069006E412610D126101C003C0E6
:1056750002C0019006E4126104D082D083D0E06BB1
:105685007008E965827003EA658360199006E3E0B6
:105695008F828E83F09006E4A3E0FAA3E0126118EE
:0556A5009006E3E0F0B7
:0156AA0022DD
:1059BA00126101C003C002C0019007AAE0FCA3E083
:1059CA00F9D082D083D0E064017008E9658270035F
:1059DA00EC65837003FF802F9007ACE0FBA3E475AE
:1059EA00F001120E65A9F0FA120D90FF126101740E
:1059FA00019007F36B7008E965827003EA658370AA
:075A0A00069007AC12610DCC
:015A11002272
:105F0800126101C003C002C0019007AAE0FCA3E02F
:105F1800F9D082D083D0E064017008E9658270030B
:0F5F2800EC65837003FF8007126101120D90FF7B
:015F37002247
:106280007B017A0779B39007ACEBF0A3EAF0A3E9BE
:05629000F0126118226C
:104200009007A8E5B0F0E05438FF9007B2E0FE6FE9
:104210006017EE6FFC543060069007B07410F09099
:1042200007A8E054389007B2F09007B0E060371468
:10423000F070339007A8E0FF9007B1E06FFCC2AFC9
:1042400030E409EF20E4057F10125630EC30E50C25
:104250009007A8E020E5057F20125630D2AF9007E6
:10426000A8E09007B1F0851215E5B020E2047F01C7
:1042700080027F008F12E512602CE5157004F5189E
:10428000F5190519E51970020518D39420E518945D
:1042900003403A9007AFE070057F40125630900718
:1042A000AF7401F08027E5127023E515601FD3E598
:1042B00019940AE5189400400FE5199420E5189424
:1042C0000350057F04125630E49007AFF0851617AF
:1042D000E5B020E3047F0180027F008F16E51660C1
:1042E0002BE5177004F513F5140514E51470020599
:1042F00013D39420E513940340399007AFE0700581
:104300007F801256309007AF7401F022E5167023BB
:10431000E517601FD3E514940AE5139400400FE5F8
:10432000149420E513940350057F08125630E4904E
:0343300007AFF0E4
:014333002267
:0E1A0500E475F001020E65EEF0A3EFF0A322EF
:0B635100AF01AE027C00E4FD025962C7
:05629500900718EDF078
:10629A00AF01AE027C00E4FDE090071DF002572337
:10578F00900712121A0CECF0A3EDF0A3EAF0A3EBC2
:10579F00F0900716E07002A3E06046900712E0FE5B
:1057AF00A3E0AA06F97B01A3E0FEA3E0F5828E83B6
:1057BF00E0FD126295900717E024FFF0900716E0C6
:1057CF0034FFF0900715E004F07006900714E00422
:1057DF00F0900713E004F070B8900712E004F08027
:0257EF00B022E6
:08636500E4900000F0A3F02217
:10601600900000E0FEA3E0AA06F97BFF1263519010
:106026000000E0FEA3E0FF7C007D027B007A041204
:0A603600578FE4900000F0A3F02261
:0D549A0090070DEDF090070BEEF0A3EFF082
:1054A700EE54FCFE900000E0FCA3E0FD7002EE6C01
:1054B700604EED4C600312601690070BE0FEEE5451
:1054C700FCFE7F00900000F0A3EFF090070E121A89
:1054D7000C7400F0A37402F07FFF7E0390070E1296
:1054E7001A0585F082F583E493FD900710121A05DB
:1054F70085F082F583EDF0EF1F70011EEF4E70DC33
:1055070090070DE0FF90070BE0FCA3E0FDEC5403D0
:0D551700FC74022DF58274003CF583EFF06A
:015524002264
:105DF0009006F4121A0CEBF0A3EAF0A3E9F0900677
:105E0000F974FFF5F0120E6545F0601E9006F4126D
:105E10001A05AFF0FE9006F6E0FBA3121A05A9F0F2
:0B5E2000FA120D90FD12549A80D4225B
:105B98009006E37427F0A37410F09006E374FFF501
:0F5BA800F0120E65FED3E5F09400EE940050EB82
:105BB7007D017F041257F11262531262E712633BB1
:105BC70012634612626A75F704125D767FD77E0507
:0A5BD7001260DDE4F58475D10322AD
:1057F100AE8475840F758C20E4F58475EF0675848D
:105801000F758A83F59775840F758904F58475B7CB
:105811003075840F4389018D8D758F018F8EFDFC4D
:105821000DBD00010CE4B505F7ECB401F3438902A9
:10583100E58920E4120DEDAA0470010C14D3940043
:10584100EA6480948140E9759702E4F58AAF068F96
:0158510084D2
:015852002233
:10625300AF8475840F75E10375E3C043A50175A68B
:06626300FF75A4E78F8423
:016269002212
:1062E700E4F584759A73759D1843E60175F801C244
:0262F700FF2284
:10626A00AF84E4F584F5BA75BC9875E88143E70212
:05627A0043F7028F84D0
:01627F0022FC
:1060DD00AD84758402E4F5C875C908C39FFFE49EBD
:1060ED00F5CB8FCA74FFF5CDF5CC43E704D2CAAF1B
:0360FD00058F8488
:01610000227C
:04638700000402010B
:105E9C00FCA3E0FDEC4EFFEDCF900869F0A3EFF012
:105EAC0022E054FEFEA3E0547F4480FF900869EE8C
:105EBC0022FEA3E0547FFFEE440190086922900873
:085ECC0069E0FEA3E054F0229E
:103DC900300606900867E08004A207E4335401C472
:103DD9003333335480FE900869E0547F125E9C901F
:103DE9000867E0FDC3135403906387935407C454D1
:103DF900F0FE900869E0548FFAA3E0FBEA4EFFEB6E
:103E0900125EA4ED131313540725E0FE900869E030
:103E190054F1125E9C900867E0FFC413135403F930
:103E290074017E00A801088005C333CE33CED8F9CA
:103E39005407C4F8540FC868FFE4C454F048FE900E
:103E49000869E0FCA3E0548FFDEC4EFEED4FFFEE58
:103E5900125EA5900407E0FD7C00C39455EC940024
:103E69005007125ECA440C8012C3ED94AAEC940068
:103E7900125ECA5004440980024403FF900869EEA7
:103E8900F0A3EFF0E964027028900838E0FCA3E0A1
:103E9900D39400EC94804008900869125EAD8027A5
:103EA900C3EC9480900869E054FE5027125EBD80EF
:103EB90016E97019E50C90086930E705125EAD80C6
:103EC90006E054FE125EBDF0A3EFF0800C90086985
:103ED900E054FEF0A3E0547FF0C287C285E4FD9070
:103EE9000869E0FEA3E0A805088005CEC313CE1338
:073EF900D8F9139286D2856F
:103F0000E49006E3F0A3F09006E4E004F07006907D
:103F100006E3E004F09006E3E07004A3E0640170BF
:013F2000E6BA
:023F2100C28557
:103F2300E49006E3F0A3F09006E4E004F07006905A
:103F330006E3E004F09006E3E07004A3E06401709C
:013F4300E697
:073F44000DEDB4109FD287C0
:013F4B002253
:0450640041085E00A1
:08636D007F0212585302632D58
:065F3800126375EF602703
:105F3E0090073E7408F0A37457F0125F6890073E06
:105F4E00E475F001120E6585F082F583EFF01263B1
:075F5E007BEF70E67F0122DA
:035F65007F002298
:106122009006E3EFF0A3EDF07F0A1258539006E3D6
:10613200E0FF1258539006E4E0FF12585302632D19
:1062AA009006E3EFF07F2F1258539006E3E0FF12B7
:0562BA00585302632DA2
:1062BF009006E3EFF07F301258539006E3E0FF12A1
:0562CF00585302632D8D
:10623B00000002AB055508000AAB0D55100012AB60
:08624B00155518001AAB1D5592
:07506800C10D420863003294
:10617F00900749E4F0A322900742E0FBA3E0FAA3C3
:0D618F00E0F92290074512101A90074522F2
:10457800EF75F00C84E5F0FD12617FEDF0EF75F05A
:104588000C8424FFFFE434FFFE900749E0FCA3E01D
:10459800FDEC6003024640EDB40C004003024640C7
:1045A8009045AFF82828730245D30245DC0245E45C
:1045B8000245EC0245F40245FC02460402460C02A0
:1045C800461402461C02462902463412617F7403CF
:1045D800F002464412617F7404F0806012617F74B7
:1045E80005F0805812617F7406F0805012617F7464
:1045F80007F0804812617F7408F0804012617F7470
:1046080009F0803812617F740AF0803012617F747B
:104618000BF08028E4900749F0A3F00FBF0000805A
:104628001B12617F04F00FBF0000801012617F74BD
:1046380002F00FBF00008004E4FEFF22EF7F00C4F9
:104648003354E0FEE4FCFD126192E0F8A3E0F9A324
:10465800E0FAA3E0FB90074AE025E0FF900749E075
:1046680033FE743B2FF58274623EF583E493FE7447
:104678000193FFE4FCFDEB2FFFEA3EFEED39FDEC74
:0C46880038FC126192A3A3E0FEA3E0FF47
:014694002203
:0B479E0090073EEBF0A3EAF0A3E9F067
:1047A900900001120DA9900741F0540FFD90086681
:1047B900E05403FF74087E00A807088006CEA2E72C
:1047C90013CE13D8F8FFEF5D24FF9205E92402F90F
:1047D900E43AFA900742EBF0A3EAF0A3E9F0900774
:1047E90041E054F02450602124D0605524506003E6
:1047F9000248A42005030248A4126186120D90FF05
:1048090012457812635CD20D222005030248A412D6
:104819006186120D90641F60030248A49000011282
:104829000DA9FF7E00900863EEF0A3EFF0D3943357
:10483900EE94004066E024FFF0900863E034FFF056
:104849002230055790073E126189900003120DA985
:1048590025E0900861F0A3E4F0900002120DA9751B
:10486900F004A4FF900861E045F0FEA3E04FFF903B
:104879000861EEF0A3EFF02401FFEE348090085FA9
:10488900F0A3EFF090085FE0FEA3E07803CEA2E783
:0B48990013CE13D8F8F0EE90085FF08B
:0148A40022F1
:074C93009006F0EFF0A90507
:104C9A00C20120C3FD20C5FAC2C4D2C5E4FFFD305B
:104CAA00C3FD30C3FDE5C154F8FC64086004ECB4EC
:104CBA001013EFB40105EB44018003EB54FEF5C277
:104CCA007D01024D61ECB4180B89C27D02C2C4C2D7
:104CDA00C5024D61ECB420028045EC6428703CEDBD
:104CEA00B4020E9006F0E0F5C27D03C2C5C2C480CC
:104CFA0066EDB4031B300008D2C57F01C2C48057D9
:104D0A009006F3E0F5C2C2C57D04E4FFC2C4804741
:104D1A00ED64047042D2C47D05803CECB4300AD202
:104D2A00C4D2C57D08E4FF802EECB438028024EC9E
:104D3A00B44006C2C2C2C5801EECB448028014EC5C
:104D4A00B450028004ECB4580AD2C47D07AEC2C281
:104D5A00C28004D2C4D2C5C2C3ED64076008ED6440
:084D6A00056003024CACAF062A
:014D7200221E
:02506F00C10975
:105A12009007FDE475F001120E6585F082F5832290
:105A22009007FD7408F0A37413F0229007F9E0FFC9
:105A3200A3E09007F5229007F9E0FEA3E0FF9007AC
:105A4200F5227E087F279007F5E022E0F5C2900755
:105A5200F5E06E229007F6E004F0229007F5E004EC
:025A6200F02230
:10620900AF84E4F584C2C343E60243F60275C301D1
:0862190075C04475CF8F8F841E
:01622100225A
:105D76007E077FFF9007F7EEF0A3EFF09007FBEEAC
:105D8600F0A3EFF09007F3EEF0A3EFF07E087F1399
:105D96009007F9EEF0A3EFF09007FDEEF0A3EFF019
:0D5DA6009007F5EEF0A3EFF0C208026209CD
:106069009007FB125A15EFF09007FB125A15EDF045
:106079009007FBE0B4080FA3E0B4130A9007FB7480
:0760890007F0A374FFF022F1
:0D632D00AF84E4F584C208C2C4D2C58F84D9
:01633A002240
:1058530020082FD208125A1274FFF07C087D27907B
:1058630007FDE0B50408A3E0B50503125A22125A56
:1058730012E4F09007FDE0B50408A3E0B5050312B8
:105883005A22125A12E4F09007FDE0B40808A3E08C
:10589300B42703125A22125A12EFF09007FDE0B414
:0D58A3000808A3E0B42703125A227F012257
:105F95009007F7E0FCA3E0FD9007F3E0B50408A344
:105FA500E0B505037F00229007F7E0FCA3E0F5824A
:0C5FB5008C83E0B507037F01227F0022EF
:105F68009007F8E004F070069007F7E004F0900757
:105F7800F7125A15E0FF9007F7E0B4080FA3E0B452
:0C5F8800130A9007F77407F0A374FFF0F1
:015F940022EA
:066375007FFF125F95227C
:06637B00E4FF125F952211
:10604000125A38E0FCA3E0FDB5071BECB50617902B
:1060500007FDE0FEA3E0FFEDB5070BECB50607205A
:09606000C5047F0180027F0022CB
:031A1800023C127B
:103C1200C0E0C0F0C083C082C0D075D000C000C078
:103C220004C005C006C007E5C154F81210633D8DFB
:103C3200003C6D083C6D103C9E183CCD203CD328C6
:103C42003D38303D3D383D47503D47583D53603D3E
:103C520049683D53703D49783D47803D62883D4704
:103C6200903D62983D75A000003DB2C2C5125A5601
:103C72007003125A5D125A44B5060BA3E0B507064B
:103C82009007F5125A259007F5125A15125A4D70DF
:103C920003A3E06F6003023DB2023D2F125A567039
:103CA20003125A5D125A44B5060BA3E0B5070690FB
:103CB20007F5125A259007F5125A15125A4D70033C
:103CC200A3E06F6003023DB2023D2F125A2DCF8056
:103CD200169007FD125A3BE0FCA3E0FDB50713EC7A
:103CE200B5060F9007F9EEF0A3EFF0C2C5D2C402F9
:103CF2003DB28D828C83E0B4FF07C2C4D2C5023DBF
:103D0200B2125A567003125A5D125A44B5060BA3E8
:103D1200E0B507069007F5125A259007F5125A15D5
:103D2200125A4D7003A3E06F6003023DB29007F593
:103D3200125A25023DB2125A2D802F125A2DCFF05F
:103D4200A3EFF0806B8010125A2DCFF0A3EFF0D2C8
:103D520009ADC27FFF8004ADC2E4FF1260698050EA
:103D62009007F3E0FFA3E09007FBCFF0A3EFF0D2C0
:103D7200C4803D9007FBE0FFA3E09007F3CFF0A3E0
:103D8200EFF030092BD2C5C2098025125A38EEF065
:103D9200A3EFF09007F3E0FDA3E09007FBCDF0A3C3
:103DA200EDF0D2C4A3E06E7003A3E06F6002D2C54F
:103DB200C2C3D007D006D005D004D000D0D0D08264
:073DC200D083D0F0D0E03205
:10630B00900867E054FEF054F9F054C7F0543FF096
:01631B00225F
:1062D400900867E020E0044401F022900867E0544D
:0362E400FEF022A7
:10609000900867E0FFC313FEEF54F9FFEE045403CA
:1060A00025E04FFFF0E0C3135403FEEF54F9FFEE79
:0760B000540325E04FF0222C
:1061B900900867E0FF131313541FFEEF54C7FFEE57
:0B61C90004540733333354F84FF02226
:105FC100900867E0FFC413135403FEEF543FFFEE44
:105FD100045403C4333354C04FF0E0FFC4131354CB
:0B5FE10003D394024004EF543FF02271
:104334000204FFFFFFFF03050100070906080AFF47
:10434400FFFFFF0DFF0B0E0C00010002000400082C
:1043540000100020004000000102020304040506CE
:1043640007070809090A0B0C0C0D0E0E0F1011118A
:10437400121314141516171718191A1A1B1C1D1EBC
:104384001E1F202121222324252526272829292AE6
:104394002B2C2D2D2E2F3031323233343536373706
:1043A40038393A3B3C3D3D3E3F404142434344451E
:1043B400464748494A4B4B4C4D4E4F50515253542B
:1043C4005556565758595A5B5C5D5E5F606162632F
:1043D4006465666768696A6B6C6C6D6E6F70717228
:1043E4007374757778797A7B7C7D7E7F8081828314
:1043F4008485868788898A8B8C8E8F9091929394FA
:10440400959697989A9B9C9D9E9FA0A1A3A4A5A6D0
:10441400A7A8A9ABACADAEAFB0B2B3B4B5B6B7B99B
:10442400BABBBCBDBFC0C1C2C4C5C6C7C8CACBCC59
:10443400CDCFD0D1D2D4D5D6D8D9DADBDDDEDFE109
:10444400E2E3E5E6E7E8EAEBECEEEFF0F2F3F5F6AB
:06445400F7F9FAFBFDFE82
:10507100C10E420402000042063700004104040050
:10164E00E4F556E55225E0FFE55133FE744C2FF5D7
:10165E008274433EF583E493FE740193FFF555E5E2
:10166E0057540FF553E55854F0F55475C30385538D
:10167E00C28554C1759208759100C281C28185964A
:10168E0053859554745A2554F58274433553F58316
:10169E00E493755700F55875C3018557C28558C137
:1016AE0022E557540FF553E55854F0F55475C3031E
:1016BE008553C28554C1759208759100C281C2814D
:1016CE00859653859554745A2554F5827443355333
:1016DE00F583E493755700F55875C3018557C28598
:1016EE0058C122FBAA06E0FEA3E0FFEF2BFFEE3A65
:1016FE00FEE433FDE433FCA312101AE47FFF7EFFF9
:10170E00FDFC22759200759140C281C2818594576D
:10171E00859358E5584256E557425522EF75F01716
:10172E00A4241DF582E5F03404F58322C281C28122
:10173E00859457859358E5584256E5574255755747
:10174E003775580075C3018555C28556C1855792A8
:10175E00855891C281C281859657859558223480CD
:10176E00AD07FCE0C313FEA3E01375C30E8CC28D50
:10177E00C18E92F59175C27F75C1FF2290072BE045
:10178E0075F017A42419F582E5F03404F58322FDD3
:10179E00ECC4F854F0C868FAEDC4540F48FBECC31F
:1017AE0013FEED132BFDEE3AFCE01313543F7E00B7
:1017BE002D22E0FEA3E0FF8E928F91C281C281C2E4
:1017CE00812275580075C3018555C28556C185574E
:1017DE0092855891C281C28185965785955822E08F
:1017EE00F8A3E0F9A3E0FAA3E0FB228508C285097D
:1017FE00C18510928511912275F017A42409F582E6
:10180E00E5F03404F58322759200759108C281C209
:10181E0081859651859552E552640745512290086F
:10182E0042E0C313FEA3E01322900860E02FF552AE
:10183E0090085FE03EF55122900729E0FEA3E0FFFD
:10184E0022E0FCA3E0FDA3E0FEA3E0FF22A4241E01
:10185E00F582E5F03404F58322E0FEA3E07803225E
:10186E0085085785095875C30322A3A3E0FFA3E09B
:01187E002247
:105DB300E49006E3F09006E3E0FB12178E12102640
:105DC30000000000EB12172BE4F0FF9006E3E01253
:105DD300180675F002EF121057E4F0A3F00FEFB4BA
:0C5DE30008E99006E3E004F0E0B40FC90A
:015DEF002291
:0B187F00900728EFF0A3ECF0A3EDF0C1
:10188A00A2AF9203900728E0FF9043349390072B6E
:10189A00F0F4703EEFB4120F900729E0FCA3E0FDCC
:1018AA00E4FF1250AA8017900728E0B4140DA3E0B1
:1018BA00FCA3E0FD7F011250AA800312184690078C
:1018CA0028E025E02478F582E43407F583EEF0A3D6
:1018DA00EFF012178AC083C08212184FC006C007E1
:1018EA0090072BE0FF121806C083C08212172AE065
:1018FA005407D082D08375F002121057E0FEA3E09D
:10190A00FBAA06D007D006C3EF9BFFEE9AFEED9422
:10191A0000FDEC9400FCD082D08312101A12178AB0
:10192A00C083C0821217ED121846E4FCFDEB2FFFAC
:10193A00EA3EFEED39FDEC38FCD082D08312101A53
:10194A0090072BE0FB12178E12184F7803120FBF65
:10195A0075F017EB12185BEEF0A3EFF0121846A31E
:10196A00E0FD121806C083C08275F017ED12172E1B
:10197A00E0D082D08375F002121057EEF0A3EFF098
:10198A0090072BE0FF12172BE004F012172AE054FD
:10199A0007F0200E6590072BE0FF12172BE0705A14
:1019AA00900403E004F07006900402E004F090074B
:1019BA002BE0FE75F01712185BE0FCA3E0FDEE25A4
:1019CA00E024A2F582E43406F583ECF0FCA3EDF002
:1019DA00FDEF25E02484F582E43406F583ECF0A3D8
:1019EA00EDF0C3900403E0943C900402E064809418
:0A19FA00804007D20EE4FF126222C3
:011A040022BF
:104F1A00900404E0FF75F00584E5F0147003024F75
:104F2A00D1147003024FD6147003024FDB147003BE
:104F3A00024FE024046003024FE3EF75F00784E5B3
:104F4A00F0B407004003024FE3904F5AF828287341
:104F5A00024F6F024F74024F83024F79024F7E0253
:104F6A004F88024FB2125B4E806F125CF6806A1253
:104F7A005D368065125CB38060125A64805B90086B
:104F8A005EE07055125F38EF604F900858E030E7E6
:104F9A000F900867E030E04190085E7402F08039B3
:104FAA0090085E7401F0803190085EE06402702916
:104FBA00900867E030E0227B017A08795712479E11
:104FCA00E490085EF08012124695800D1255AB806F
:0F4FDA000812445A80031240B8900404E004F017
:014FE90022A5
:045C2900AD07AC0611
:105C2D00900844E0FEA3E07806CEC313CE13D8F956
:105C3D002401FFEE34FEFED3EF9400EE64809480D9
:105C4D00400FEF2DFDEE3CFC30E7127C7F7DFF8099
:105C5D000CEF2DFDEE3CFC30E703E4FCFDAE04AF94
:015C6D000531
:015C6E002213
:1040B800900867E030E03B900863E0FEA3E0FF640F
:1040C800324E6022EF24CEFFEE34FFFEEF7802C3BB
:1040D80033CE33CED8F9FDAC0612182C2DFFEE3CAA
:1040E800FE121837802312182CFF121837AF52FE11
:1040F8008010900842E0C313F551A3E013F552FF76
:10410800AE51125C298E518F52900849E02400F577
:1041180058900848E03480F557900846121867CE42
:10412800C313CE13D8F9F5568E55900772E0256063
:10413800FF900771E0355F6480F5538F549007A0B6
:10414800E0FCA3E09007A012179DF55AEE3CF55944
:1041580030E70675597F755AFFC3E55A955CF55ADD
:10416800E559955BF55930E705E4F559F55A900896
:1041780067E0FF30E015900863E07004A3E0643264
:104188006009E4F553F554F559F55A75C30E85538E
:10419800C28554C18555928556918557C28558C1A7
:1041A800855992855A911217838551928552911299
:1041B80017C985CF0A85CE0BEF131313540730E0C8
:1041C8002C75C30E121783850A92850B91850CC234
:1041D800850DC1900405121867CEC313CE13D8F904
:1041E8008E92F5911217C985CF0A85CE0BE50A3054
:0741F800E705E4F50AF50BF1
:0141FF00229D
:1055AB00850A57850B58C3E557648094805005E4F2
:1055BB00F557F55875C3031216EA759200759108E5
:1055CB00C281C281859651859552E552640745513A
:1055DB007018F5567555401216AF759200759140BF
:1055EB0012173A85571085581122E4F556E55225C6
:1055FB00E0FFE55133FE744C2FF58274433EF58387
:10560B00E493FE740193FFF5551216AF8E928F91B2
:10561B0012173AE557A2E713F557E55813F55885D6
:04562B005710F5110E
:01562F002258
:10445A00900867E0C4131354031460361460782478
:10446A0002600302457712186E1216A81218157008
:10447A0011F55675554012166D121711755702022D
:10448A0044B512164E8E928F911217177557020263
:10449A0044CC12186E1216A81218157018F5567513
:1044AA00554012166D1217117557371217D08557C6
:1044BA000E85580F2212164E8E928F91121717756B
:1044CA0057371217D0E557A2E713F557E55813F5F2
:1044DA005885570EF50F22E50925E0F509E5083359
:1044EA00F50830E72063088075C30E1217F9121712
:1044FA00F91217F91217831217FF1217C985CF0E6F
:10450A0085CE0F804575C30EC374FF9509FF747F6E
:10451A009508F5C28FC11217FF1217C985CF0E85EC
:10452A00CE0FE50FAE0E7802CEC313CE13D8F9FD27
:10453A00AC06E50EC313FEE50F132DFFEE3CFEC3DA
:10454A00E5119FF50FE5109EF50ED3E50F9480E572
:10455A000E941B4007750E1B750F8022C3E50F943E
:0D456A001CE50E94005006750E00750F1C28
:014577002221
:1046950090083AE0FEA3E07806CEC313CE13D8F90E
:1046A5002401FDEE34FCFC90083812182F2DFFEC88
:1046B5003EFE900638E02FF552900637E03EF55164
:1046C500900867E0C3135403FFBF033074402552BD
:1046D500F55274053551F551900775E0FEA3E07864
:1046E50005CEC313CE13D8F9FFC3E5529FF552E5A6
:1046F500519EF55130E705E4F551F55290083FE03C
:104705002400F55890083EE03480F55790083C1297
:104715001867CEC313CE13D8F9F5568E5590076C8E
:10472500E02562FF90076BE035616480F5538F5497
:1047350090079CE0FCA3E090079C12179DF55AEEAC
:104745003CF55930E70675597F755AFFC3E55A950B
:104755005EF55AE559955DF55930E705E4F559F5E6
:104765005A75C30E8553C28554C185559285569198
:104775008557C28558C1855992855A9112178385E7
:1047850051928552911217C985CF0885CE09E50842
:0847950030E705E4F508F50921
:01479D0022F9
:105B4E0090082EE0C313FFA3E01390073ECFF0A3FF
:105B5E00EFF090082DE02400FF90082CE090077ED7
:105B6E0012176C90073E1217C0900405E5CFF0A3F4
:105B7E00E5CEF0E02401F0900405E034FFF0E030D3
:095B8E00E707E4900405F0A3F020
:015B970022EB
:105A6400900830E0C313FFA3E01390073ECFF0A3E8
:105A7400EFF0900833E02400FF900832E090077CB8
:105A840012176C90073E1217C0900631E5CFF0A3B1
:105A9400E5CEF0900631E030E707E4900631F0A35C
:0E5AA400F0900632E025E0F0900631E033F09D
:015AB20022D1
:105CF600900840E0FFA3E090073ECFF0A3EFF090BE
:105D06000796E0FEA3E090073E1216F190074012B8
:105D160017EDD3120FAE400974FF900407F0A3F0FD
:0F5D260022900740121878900407CFF0A3EFF0F7
:015D3500224B
:105D3600900834E0FFA3E090073ECFF0A3EFF09089
:105D46000782E0FEA3E090073E1216F1900740128C
:105D560017EDD3120FAE400974FF900633F0A3F08F
:0F5D660022900740121878900633CFF0A3EFF089
:015D7500220B
:105CB300900836E0FFA3E090073ECFF0A3EFF0900B
:105CC3000780E0FEA3E0FBAA0690073E1216F490BD
:105CD30007401217EDD3120FAE400974FF9006353B
:105CE300F0A3F022900740121878900635CFF0A366
:025CF300EFF0D0
:015CF500228C
:09635C00900842EEF0A3EFF022DC
:10631C00FF00000000000000000000000000000072
:01632C000070
:06508100C10A41082700EE
:103A360090C00175F01FED121057EC75F01FA4250C
:103A460083AF829006EBF0A3EFF09006E3E09006DA
:103A5600E875F01FA42401F974C035F0FA74FFF07C
:103A6600A3EAF0A3E9F0229006E8A3E475F00112B8
:103A76000E659006EBFEAFF0E475F001120E65855B
:103A8600F082F583E49322900827E075F01FA424C2
:103A960001F582E5F034C022900867E0FF5406FE87
:103AA60090082BE054F94EFEF0EF5438FFEE54C761
:103AB6004FFFF0900867E090082B54C0FEEF543F8C
:103AC6004EF022A3E0FCA3E0FDA3E0FEA3E0FF7816
:103AD60004020FBFAF82FE7A08792B7B019006F9AC
:103AE600E4F0A322FBE0FEA3E0FFC3E49FFF7480A3
:103AF6009EFE3395E0FDFCEB2FFFEA3EFE22E4330B
:103B0600F0A3E58EF0A3E589F0A3E58DF0A3E58BA0
:103B1600F0A28EE433A3F0900829E0FF22E0F8A398
:103B2600E0F9A3E0FAA3E0229007A0E0FCA3E0FD01
:103B3600ECC4F854F0C868FAEDC4540F48FB22E010
:103B460024FFFFE434FFFE9006E4E0FCA3E0FD2240
:103B56009006E3A3E475F001020E65FDEDFFEEF0BD
:103B6600A3EFF0C2AF900827740FF022900709E088
:103B7600FCA3E0FDC3941FEC9400227EC37FA37BCD
:103B8600007A00795B2224FFFEE434FF9006E4F01D
:103B9600A3CEF022C39006E7E0941F9006E6E094D9
:103BA6000022E075F01FA42401F974C035F0FA2252
:103BB600EF25E0242CF582E43408F58322E0FCA30B
:103BC600E0FFECFD90082AE0FB22E4900709F0A351
:103BD600F0227F00FEF0A3EFF0900828E02274E8C0
:103BE6002DF582E43406F58322ED39FDEC38FC022E
:103BF600101AE93DFDE83CFC02101A9FEE6480F8BD
:0C3C0600EC64809822900709E004F02292
:1060B70090082BE0FF5406FE900867E054F94EFE67
:1060C700F0EF5438FFEE54C74FFFF090082BE090E5
:0660D7000867123AC02226
:04638B00123A9E2202
:10590900123A9EE4FFEF600D64036009EF640960D9
:1059190004EFB40E0B123BB67480F0A3E4F08007D9
:10592900123BB6E4F0A3F00FEFB40FD9126365E4AC
:105939009006E9F09006E9E0FFC3941E501875F04F
:105949001FEF123A94123ADA741FF0125DF09006C2
:09595900E9E004F080DE026016B2
:105ED4009006E77402F0E4A3F01263657EC07F00CD
:105EE4007A0679E7123AE104F0125DF07EC37FABE3
:105EF4007B017A0679E8123AE304F0125DF012604D
:045F0400160259091F
:10619C00200A1730060C900867E030E00712636D98
:0D61AC008002D2079008657401F0D20A222B
:1048A50078E47C067D017BFF7A63791D7E007F10AD
:1048B500120D6AA2AF9200D2AF300EFDC2AFE490E6
:1048C50006E3F09006E4123B23FBC000C002C003E0
:1048D500123B2EECC313FEED132BFDEE3AFC9007B5
:1048E500A0E01313543F7E002DFFEE3CFEE4FCFDDB
:1048F500D003D002D000123AFD9006E4123BEF90AF
:1049050006E8123B23FBC000C002C003123B2E90F9
:10491500079CE0C313FEA3E0132BFBEE3AFAEC135E
:1049250013543F7E002BFFEE3AFEE4FCFDD003D08E
:1049350002D000123AFD9006E8123BEF9006EC1209
:104945003B23900771123AEA9006EC123BF8900669
:10495500F0123B2390076B123AEA9006F0123BF8EF
:104965009006E3E004F0E0641060030248C8900696
:10497500E4123ACA8E5B8F5C123AC98E5D8F5E1265
:104985003AC98E5F8F60123AC98E618F6212636574
:10499500123B81123AE37408F0125DF0126016A220
:0349A5000092AFCE
:0149A80022EC
:1054090090C3ABE493700302549190C000E4936499
:03541900026031FD
:10541C00A2AF9200125ED4D2AF300EFDC2AF1263B7
:10542C0065123B81123AE37408F0125DF0126016BB
:0F543C007A63791C7B01E4FD126295A20092AFA6
:02544B0080449B
:10544D007BFF7AC379A3AF01AE027DFF7C0090068E
:10545D00E312101A9006E3A3A3E0FEA3E0FFE4FD20
:10546D00FC9006E312101A123B859006E3E0FCA3B4
:10547D00E0FDA3E0FEA3E0FF900733E4F0A3740882
:04548D00F01258B011
:095491001261EFE4900827F022FB
:10614200123A8DF583AF82FE7C00E4FD7B017A0872
:0F615200792B900733F0A3741FF01258B0C20AD4
:01616100221B
:1062F900126365123A8D123ADA741FF0125DF002D8
:0263090060161C
:066381001262F9C20A22BB
:0261D400AD0715
:1061D600A2AF9200C2AF12638B900827EDF0126354
:0861E600811261EFA20092AFEB
:0161EE00228E
:10622200A2AF9204C2AF900827EFF012614212604F
:08623200B71261EFA20492AF64
:01623A002241
:1051670090084DE0FB90084BE0FED39B4050EE12B9
:105177003B8CEB149006E3F090084A123B45D312A0
:105187003C014003025218123A36E49006E6F0A3B7
:10519700F0123A6D12521970069006E6E004F0120A
:1051A7003B9A40ED1260169006E5E004F070069019
:1051B70006E4E004F09006E3E004F002517F900873
:1051C7004AE0123B8C90084CE0149006E3F09008FC
:1051D7004B123B45C3123C014037123A36E4900666
:1051E700E6F0A3F0123A6D12521970069006E6E047
:1051F70004F0123B9A40ED1260169006E5E024FF9A
:10520700F09006E4E034FFF09006E3E014F002517A
:01521700D5C1
:0C52180022FD12549A9006E7E004F022F8
:104E470090084BE014900707F090084DE014900786
:104E570008F090084AE014FF900707E0D39F40034B
:104E6700024F0EA3123A90AF82FE123BD0123B7252
:104E770050210FEFAA0670010E14F5828A83E4937E
:104E8700FB123BE4EBF090070AE004F070DF123C02
:104E97000B80DA900708E09006E3123A579007076D
:104EA700123A90AF829006E6F0A3EFF0123BD012D1
:104EB7003B569006E6123A7B124F0F7003123C0BDB
:104EC700C390070AE0941F900709E0940040E09020
:104ED7000707123BA89006E3123A63123BD0123B36
:104EE700725014123B56FEAFF0123BE4E0124F0F24
:104EF70070EC123C0B80E7126016900707E004F095
:074F0700A3E004F0024E5983
:0C4F0E0022FD12549A90070AE004F022E1
:10552500A2AF9006E3123B049006E9E4F0A3EFF086
:10553500E09006E9123BD89006E9123B61126365DB
:10554500900827123BA89006EB123A63E4A3F0906B
:1055550006E9123BC3E49006F3F0D200124C939097
:1055650006EFEFF0FD9006EB123B59FEAFF012543B
:105575009A9006EAE004F070069006E9E004F090DF
:1055850006EEE004F0E0C3941F40C41260169008D4
:1055950027E004F0E0C3941E40A3125D769006E375
:0555A500E024FF92AFBD
:0155AA0022DE
:10537600A2AF9006E3123B049006EBE4F0A3EFF035
:10538600E09006EB123BD89006EB123B61900827A3
:10539600E0FFC3941E506075F01FEF123A94AF827F
:1053A6009006EDF0A3EFF0E49006E9F0A3F0900686
:1053B600EB123BC39006ED123A7E9006F3F0C20064
:1053C600124C939006ECE004F070069006EBE004B5
:1053D600F09006EAE004F070069006E9E004F0C3F7
:1053E6009006EAE0941F9006E9E0940040C0900819
:1053F60027E004F0025393125D769006E3E024FF63
:0254060092AF63
:015408002281
:10508700C10F1E22000900080000000600010007EA
:10509700000C000A000D000B000E0015001700138E
:0250A7000016F1
:104BA0009006E3E025E0242CF582E43408F5832226
:104BB000C3EF9BFFEE9AFEED9400FDEC9400FC9099
:104BC00006E812101AE47F80FE9006E8FDFCE0F88B
:104BD000A3E0F9A3E0FAA3E0FBD3020F98F8900654
:104BE000E3E025E025E02448F582E43406F583225D
:104BF0009006E3E025E02484F582E43406F5832280
:104C000074FF7F80FEFDFC9006E8E0F8A3A3A3E01C
:104C1000C3020F98E0FCA3E0FDA3E0FEA3E0FF12B7
:104C20000E7BE47BFF7A0FF9F822E0FEA3E0FFC3DE
:104C3000EF9BFFEE9AFEE49400FDE49400FC2278E2
:104C400004120FD28E4F8F50900867E0C413135494
:104C5000036402229006E3E02439F582E43406F589
:104C6000832225E024C0F582E43406F58322E0C4E3
:104C7000F854F0C8682225E024A2F582E43406F551
:104C800083229006E4A3A3E0FEA3E022A3E0C454A1
:034C90000F4822A8
:1061EF00E4FFEF124BA4E0FCA3E0FDEF124C62ECD6
:0961FF00F0A3EDF00FEFB40FE97D
:016208002273
:051089009006E3EFF00A
:10108E00900867E030E017900863E07004A3E06416
:10109E0032600B9006E3E0640B7003021388124B70
:1010AE00F0E0FEA3E0FBAA06E49006E3E075F0177D
:1010BE00A4241EF582E5F03404F583124C2A900622
:1010CE00E412101AE47FF47E019006E4124BCC4039
:1010DE000E754E01124C82240CFFEE34FE80287FDA
:1010EE000C7EFE7DFF7CFF9006E4E0F8A3E0F9A302
:1010FE00E0FAA3E0FBC3120F985018E4F54E124C21
:10110E008224F4FFEE3401FE124BF0EE8FF0120E3D
:10111E004F8007124C547403F0229006E3E0FD1248
:10112E004BF4124C6EF548124C8CF549ED124BA453
:10113E00124C6EF54A124C8CF54B9006E3E0124CB5
:10114E0076124C6EF54C124C8CF54D74392D124CAA
:10115E005AE0B54E03D38001C35003021229E54E67
:02116E00703AD5
:10117000E54D9401E54C940050067E007F0180040B
:10118000AE4CAF4DE48F438E42F541F540AE4AAFD1
:101190004BFCFD124C23120E7BAB43AA42A941A883
:0711A00040120F06124BDEA6
:0311A70002122011
:1011AA00AE4CAF4DAB07AA06C374FF9BF547740F4D
:1011BA009AF546E49400F545E49400F544C374FFB7
:1011CA00954BFF740F954AFEE4FCFD124C23120E58
:1011DA007B124BDE12101AE47F01FEFDFCAB47AA1C
:1011EA0046A945A844C3120FAE500AE4754701F553
:1011FA0046F545F544124BDEC083C082E0FCA3E00D
:10120A00FDA3E0FEA3E0FFAB47AA46A945A8441206
:09121A005C6FD082D08312101A1F
:10122300124C54E54EF0E54E706FAE48AF49AB0734
:10123300AA06F9124BDD124C14125C6F124C3F706C
:10124300559006E3E0FF6406704C200F0EEF124B3F
:10125300A4E0654FFEEE30E702D20F200F03021326
:011263002268
:10126400124BA0E0FEA3E0FFE4FCFDC006C007AE05
:101274004FAF50AB07AA06D007D006124BB05005AB
:10128400124C005003021313124BA0747FF0A3748A
:02129400FFF069
:1012960002132E021322AE48AF49AB07AA06C37447
:1012A600FF9BFB740F9AFAE49400F9E49400124B46
:1012B600DD124C14120F06C374FF9FFF740F9EFEBF
:1012C600E49DFDE49CFC124C3F70539006E3E0FF66
:1012D6006406704A200F0EEF124BA4E0654FFEEE37
:0812E60030E702D20F300F3493
:1012EE00124BA0E0FEA3E0FFE4FCFDC006C007AE7B
:1012FE004FAF50AB07AA06D007D006124BB0500521
:10130E00124C005004C20F800D124BA07480F0A33B
:02131E00E4F0F9
:10132000800C8000124BA0E54FF0A3E550F0900632
:10133000E3E0FF124BF4E0FCA3E0FDEF124C76EC8F
:10134000F0A3EDF0900867E030E003300A062006D5
:0413500037200A3404
:101354009006E3E0124C62E0FEA3E0FBAA06124B07
:10136400A0124C2A9006E812101AE47F587E02124A
:101374004BC9500D7FA87EFD7DFF7CFF124C0750AA
:041384000312619C53
:011388002242
:101A36000000000100030004000600070009000A78
:101A4600000C000E000F0011001200140015001704
:101A56000019001A001C001D001F0020002200248F
:101A6600002500270028002A002B002D002F00301B
:101A760000320033003500360038003A003B003DA6
:101A8600003E004000410043004500460048004932
:101A9600004B004C004E00500051005300540056BD
:101AA60000570059005A005C005E005F006100624A
:101AB6000064006500670069006A006C006D006FD5
:101AC600007000720073007500770078007A007B62
:101AD600007D007E008000820083008500860088ED
:101AE6000089008B008C008E00900091009300947A
:101AF600009600970099009A009C009E009F00A106
:101B060000A200A400A500A700A800AA00AB00AD93
:101B160000AF00B000B200B300B500B600B800B91F
:101B260000BB00BC00BE00C000C100C300C400C6AC
:101B360000C700C900CA00CC00CD00CF00D100D23A
:101B460000D400D500D700D800DA00DB00DD00DEC7
:101B560000E000E100E300E400E600E800E900EB55
:101B660000EC00EE00EF00F100F200F400F500F7E3
:101B760000F800FA00FB00FD00FE01000101010370
:101B86000104010601080109010B010C010E010FF8
:101B9600011101120114011501170118011A011B87
:101BA600011D011E01200121012301240126012717
:101BB6000129012A012C012D012F013001320133A7
:101BC6000135013601380139013B013C013E013F37
:101BD600014101420144014501470148014A014BC7
:101BE600014D014E01500151015301540156015757
:101BF6000158015A015B015D015E016001610163EB
:101C06000164016601670169016A016C016D016F7A
:101C16000170017101730174017601770179017A0E
:101C2600017C017D017F018001820183018401869F
:101C360001870189018A018C018D018F0190019232
:101C460001930194019601970199019A019C019DC6
:101C5600019E01A001A101A301A401A601A701A85B
:101C660001AA01AB01AD01AE01B001B101B201B4EF
:101C760001B501B701B801BA01BB01BC01BE01BF84
:101C860001C101C201C301C501C601C801C901CA1A
:101C960001CC01CD01CF01D001D201D301D401D6AF
:101CA60001D701D801DA01DB01DD01DE01DF01E147
:101CB60001E201E401E501E601E801E901EB01ECDD
:101CC60001ED01EF01F001F101F301F401F501F776
:101CD60001F801FA01FB01FC01FE01FF020002020C
:101CE60002030204020602070209020A020B020D9F
:101CF600020E020F02110212021302150216021739
:101D06000219021A021B021D021E021F02210222D2
:101D160002230225022602270229022A022B022D6D
:101D2600022E022F02310232023302340236023709
:101D36000238023A023B023C023E023F02400242A5
:101D4600024302440245024702480249024B024C42
:101D5600024D024E025002510252025402550256E0
:101D660002570259025A025B025C025E025F02607F
:101D76000261026302640265026702680269026A1E
:101D8600026C026D026E026F0271027202730274BD
:101D96000275027702780279027A027C027D027E5F
:101DA600027F028102820283028402850287028800
:101DB6000289028A028C028D028E028F02900292A2
:101DC600029302940295029602980299029A029B45
:101DD600029C029E029F02A002A102A202A302A5E9
:101DE60002A602A702A802A902AB02AC02AD02AE8D
:101DF60002AF02B002B202B302B402B502B602B733
:101E060002B802BA02BB02BC02BD02BE02BF02C0D9
:101E160002C202C302C402C502C602C702C802CA7F
:101E260002CB02CC02CD02CE02CF02D002D102D228
:101E360002D402D502D602D702D802D902DA02DBD0
:101E460002DC02DE02DF02E002E102E202E302E479
:101E560002E502E602E702E802E902EB02EC02ED25
:101E660002EE02EF02F002F102F202F302F402F5D0
:101E760002F602F702F802F902FA02FB02FD02FE7E
:101E860002FF030003010302030303040305030621
:101E9600030703080309030A030B030C030D030ED0
:101EA600030F031003110312031303140315031680
:101EB600031703180319031A031B031C031D031E30
:101EC600031F0320032103220323032403250326E0
:101ED600032703280329032A032B032C032D032D91
:101EE600032E032F03300331033203330334033548
:101EF6000336033703380339033A033B033C033CF9
:101F0600033D033E033F03400341034203430344AF
:101F1600034503460347034703480349034A034B64
:101F2600034C034D034E034F034F0350035103521B
:101F360003530354035503560356035703580359D3
:101F4600035A035B035C035C035D035E035F03608C
:101F56000361036103620363036403650366036647
:101F6600036703680369036A036B036B036C036D02
:101F7600036E036F036F03700371037203730373BE
:101F86000374037503760377037703780379037A7B
:101F9600037A037B037C037D037E037E037F03803A
:101FA60003810381038203830384038403850386F9
:101FB6000387038703880389038A038A038B038CB9
:101FC600038C038D038E038F038F0390039103917C
:101FD600039203930394039403950396039603973E
:101FE600039803980399039A039A039B039C039D02
:101FF600039D039E039F039F03A003A103A103A2C6
:1020060003A203A303A403A403A503A603A603A78D
:1020160003A803A803A903AA03AA03AB03AB03AC53
:1020260003AD03AD03AE03AF03AF03B003B003B11B
:1020360003B203B203B303B303B403B503B503B6E4
:1020460003B603B703B703B803B903B903BA03BAB0
:1020560003BB03BB03BC03BD03BD03BE03BE03BF7B
:1020660003BF03C003C003C103C203C203C303C348
:1020760003C403C403C503C503C603C603C703C716
:1020860003C803C803C903C903CA03CA03CB03CBE6
:1020960003CC03CC03CD03CD03CE03CE03CF03CFB6
:1020A60003D003D003D103D103D203D203D203D387
:1020B60003D303D403D403D503D503D603D603D75A
:1020C60003D703D703D803D803D903D903DA03DA2E
:1020D60003DA03DB03DB03DC03DC03DC03DD03DD04
:1020E60003DE03DE03DE03DF03DF03E003E003E0DA
:1020F60003E103E103E203E203E203E303E303E3B1
:1021060003E403E403E503E503E503E603E603E688
:1021160003E703E703E703E803E803E803E903E962
:1021260003E903EA03EA03EA03EB03EB03EB03EC3D
:1021360003EC03EC03EC03ED03ED03ED03EE03EE1A
:1021460003EE03EE03EF03EF03EF03F003F003F0F8
:1021560003F003F103F103F103F103F203F203F2D7
:1021660003F203F303F303F303F303F403F403F4B7
:1021760003F403F503F503F503F503F603F603F697
:1021860003F603F603F703F703F703F703F703F87A
:1021960003F803F803F803F803F903F903F903F95D
:1021A60003F903F903FA03FA03FA03FA03FA03FA43
:1021B60003FB03FB03FB03FB03FB03FB03FB03FC28
:1021C60003FC03FC03FC03FC03FC03FC03FC03FD10
:1021D60003FD03FD03FD03FD03FD03FD03FD03FDF9
:1021E60003FE03FE03FE03FE03FE03FE03FE03FEE1
:1021F60003FE03FE03FE03FE03FF03FF03FF03FFCD
:1022060003FF03FF03FF03FF03FF03FF03FF03FFB8
:1022160003FF03FF03FF03FF03FF03FF03FF03FFA8
:1022260003FF03FF03FF03FF03FF03FF03FF03FF98
:1022360003FF03FF03FF03FF03FF03FF03FF03FF88
:1022460003FF03FF03FF03FF03FF03FF03FF03FF78
:1022560003FF03FF03FF03FF03FF03FF03FF03FF68
:1022660003FF03FF03FF03FF03FF03FE03FE03FE5B
:1022760003FE03FE03FE03FE03FE03FE03FE03FE50
:1022860003FE03FD03FD03FD03FD03FD03FD03FD47
:1022960003FD03FD03FC03FC03FC03FC03FC03FC3E
:1022A60003FC03FC03FB03FB03FB03FB03FB03FB36
:1022B60003FB03FA03FA03FA03FA03FA03FA03F930
:1022C60003F903F903F903F903F903F803F803F82B
:1022D60003F803F803F703F703F703F703F703F627
:1022E60003F603F603F603F603F503F503F503F524
:1022F60003F403F403F403F403F303F303F303F324
:1023060003F203F203F203F203F103F103F103F123
:1023160003F003F003F003F003EF03EF03EF03EE24
:1023260003EE03EE03EE03ED03ED03ED03EC03EC26
:1023360003EC03EC03EB03EB03EB03EA03EA03EA28
:1023460003E903E903E903E803E803E803E703E72E
:1023560003E703E603E603E603E503E503E503E433
:1023660003E403E303E303E303E203E203E203E13B
:1023760003E103E003E003E003DF03DF03DE03DE44
:1023860003DE03DD03DD03DC03DC03DC03DB03DB4D
:1023960003DA03DA03DA03D903D903D803D803D758
:1023A60003D703D703D603D603D503D503D403D463
:1023B60003D303D303D203D203D203D103D103D071
:1023C60003D003CF03CF03CE03CE03CD03CD03CC7F
:1023D60003CC03CB03CB03CA03CA03C903C903C88F
:1023E60003C803C703C703C603C603C503C503C49F
:1023F60003C403C303C303C203C203C103C003C0B0
:1024060003BF03BF03BE03BE03BD03BD03BC03BBC3
:1024160003BB03BA03BA03B903B903B803B703B7D7
:1024260003B603B603B503B503B403B303B303B2EC
:1024360003B203B103B003B003AF03AF03AE03AD02
:1024460003AD03AC03AB03AB03AA03AA03A903A81A
:1024560003A803A703A603A603A503A403A403A333
:1024660003A203A203A103A103A0039F039F039E4C
:10247600039D039D039C039B039A039A0399039868
:102486000398039703960396039503940394039383
:102496000392039103910390038F038F038E038DA1
:1024A600038C038C038B038A038A038903880387BF
:1024B60003870386038503840384038303820381DE
:1024C60003810380037F037E037E037D037C037BFE
:1024D600037A037A03790378037703770376037520
:1024E600037403730373037203710370036F036F43
:1024F600036E036D036C036B036B036A0369036866
:10250600036703660366036503640363036203618B
:1025160003610360035F035E035D035C035C035BAF
:10252600035A0359035803570356035603550354D6
:102536000353035203510350034F034F034E034DFE
:10254600034C034B034A0349034803470347034627
:10255600034503440343034203410340033F033E51
:10256600033D033C033C033B033A0339033803377B
:102576000336033503340333033203310330032FA9
:10258600032E032D032D032C032B032A03290328D3
:102596000327032603250324032303220321032001
:1025A600031F031E031D031C031B031A0319031831
:1025B6000317031603150314031303120311031061
:1025C600030F030E030D030C030B030A0309030891
:1025D60003070306030503040303030203010300C1
:1025E60002FF02FE02FD02FB02FA02F902F802F7FE
:1025F60002F602F502F402F302F202F102F002EF31
:1026060002EE02ED02EC02EB02E902E802E702E664
:1026160002E502E402E302E202E102E002DF02DE98
:1026260002DC02DB02DA02D902D802D702D602D5D0
:1026360002D402D202D102D002CF02CE02CD02CC07
:1026460002CB02CA02C802C702C602C502C402C33E
:1026560002C202C002BF02BE02BD02BC02BB02BA77
:1026660002B802B702B602B502B402B302B102B0B2
:1026760002AF02AE02AD02AC02AB02A902A802A7EB
:1026860002A602A502A302A202A102A0029F029E26
:10269600029C029B029A0299029802960295029463
:1026A600029302920290028F028E028D028C028A9F
:1026B60002890288028702850284028302820281DD
:1026C600027F027E027D027C027A0279027802771C
:1026D60002750274027302720271026F026E026D5B
:1026E600026C026A0269026802670265026402639A
:1026F60002610260025F025E025C025B025A0259DC
:102706000257025602550254025202510250024E1C
:10271600024D024C024B024902480247024502445E
:10272600024302420240023F023E023C023B023AA0
:102736000238023702360234023302320231022FE5
:10274600022E022D022B022A022902270226022528
:10275600022302220221021F021E021D021B021A6E
:102766000219021702160215021302120211020FB3
:10277600020E020D020B020A0209020702060204F9
:1027860002030202020001FF01FE01FC01FB01FA45
:1027960001F801F701F501F401F301F101F001EF90
:1027A60001ED01EC01EA01E901E801E601E501E4D8
:1027B60001E201E101DF01DE01DD01DB01DA01D821
:1027C60001D701D601D401D301D201D001CF01CD69
:1027D60001CC01CA01C901C801C601C501C301C2B4
:1027E60001C101BF01BE01BC01BB01BA01B801B7FD
:1027F60001B501B401B201B101B001AE01AD01AB49
:1028060001AA01A801A701A601A401A301A101A093
:10281600019E019D019C019A0199019701960194DF
:10282600019301920190018F018D018C018A01892A
:10283600018701860184018301820180017F017D78
:10284600017C017A017901770176017401730171C6
:102856000170016F016D016C016A01690167016612
:102866000164016301610160015E015D015B015A62
:102876000158015701560154015301510150014EAF
:10288600014D014B014A01480147014501440142FE
:102896000141013F013E013C013B0139013801364E
:1028A6000135013301320130012F012D012C012A9E
:1028B6000129012701260124012301210120011EEE
:1028C600011D011B011A011801170115011401123E
:1028D6000111010F010E010C010B0109010801068E
:1028E600010401030101010000FE00FD00FB00FAE6
:1028F60000F800F700F500F400F200F100EF00EE3A
:1029060000EC00EB00E900E800E600E400E300E18B
:1029160000E000DE00DD00DB00DA00D800D700D5DD
:1029260000D400D200D100CF00CD00CC00CA00C92F
:1029360000C700C600C400C300C100C000BE00BC82
:1029460000BB00B900B800B600B500B300B200B0D5
:1029560000AF00AD00AB00AA00A800A700A500A428
:1029660000A200A1009F009E009C009A009900977B
:1029760000960094009300910090008E008C008BCE
:102986000089008800860085008300820080007E22
:10299600007D007B007A0078007700750073007276
:1029A6000070006F006D006C006A006900670065CA
:1029B600006400620061005F005E005C005A00591E
:1029C600005700560054005300510050004E004C72
:1029D600004B0049004800460045004300410040C6
:1029E600003E003D003B003A00380036003500331B
:1029F60000320030002F002D002B002A002800276F
:102A06000025002400220020001F001D001C001AC3
:102A1600001900170015001400120011000F000E17
:102A2600000C000A0009000700060004000300016C
:102A36000000FFFFFFFDFFFCFFFAFFF9FFF7FFF6BF
:102A4600FFF4FFF2FFF1FFEFFFEEFFECFFEBFFE914
:102A5600FFE7FFE6FFE4FFE3FFE1FFE0FFDEFFDC69
:102A6600FFDBFFD9FFD8FFD6FFD5FFD3FFD1FFD0BD
:102A7600FFCEFFCDFFCBFFCAFFC8FFC6FFC5FFC312
:102A8600FFC2FFC0FFBFFFBDFFBBFFBAFFB8FFB766
:102A9600FFB5FFB4FFB2FFB0FFAFFFADFFACFFAABB
:102AA600FFA9FFA7FFA6FFA4FFA2FFA1FF9FFF9E0E
:102AB600FF9CFF9BFF99FF97FF96FF94FF93FF9163
:102AC600FF90FF8EFF8DFF8BFF89FF88FF86FF85B6
:102AD600FF83FF82FF80FF7EFF7DFF7BFF7AFF780B
:102AE600FF77FF75FF74FF72FF70FF6FFF6DFF6C5E
:102AF600FF6AFF69FF67FF66FF64FF62FF61FF5FB2
:102B0600FF5EFF5CFF5BFF59FF58FF56FF55FF5303
:102B1600FF51FF50FF4EFF4DFF4BFF4AFF48FF4757
:102B2600FF45FF44FF42FF40FF3FFF3DFF3CFF3AAA
:102B3600FF39FF37FF36FF34FF33FF31FF2FFF2EFC
:102B4600FF2CFF2BFF29FF28FF26FF25FF23FF224F
:102B5600FF20FF1FFF1DFF1CFF1AFF18FF17FF15A1
:102B6600FF14FF12FF11FF0FFF0EFF0CFF0BFF09F3
:102B7600FF08FF06FF05FF03FF02FF00FEFFFEFD45
:102B8600FEFCFEFAFEF8FEF7FEF5FEF4FEF2FEF19E
:102B9600FEEFFEEEFEECFEEBFEE9FEE8FEE6FEE5EF
:102BA600FEE3FEE2FEE0FEDFFEDDFEDCFEDAFED93F
:102BB600FED7FED6FED4FED3FED1FED0FECEFECD8F
:102BC600FECBFECAFEC8FEC7FEC5FEC4FEC2FEC1DF
:102BD600FEBFFEBEFEBCFEBBFEB9FEB8FEB6FEB52F
:102BE600FEB3FEB2FEB0FEAFFEADFEACFEAAFEA97F
:102BF600FEA8FEA6FEA5FEA3FEA2FEA0FE9FFE9DCB
:102C0600FE9CFE9AFE99FE97FE96FE94FE93FE911A
:102C1600FE90FE8EFE8DFE8CFE8AFE89FE87FE8667
:102C2600FE84FE83FE81FE80FE7EFE7DFE7CFE7AB5
:102C3600FE79FE77FE76FE74FE73FE71FE70FE6E02
:102C4600FE6DFE6CFE6AFE69FE67FE66FE64FE634E
:102C5600FE62FE60FE5FFE5DFE5CFE5AFE59FE5899
:102C6600FE56FE55FE53FE52FE50FE4FFE4EFE4CE5
:102C7600FE4BFE49FE48FE46FE45FE44FE42FE4130
:102C8600FE3FFE3EFE3DFE3BFE3AFE38FE37FE357B
:102C9600FE34FE33FE31FE30FE2EFE2DFE2CFE2AC5
:102CA600FE29FE28FE26FE25FE23FE22FE21FE1F0D
:102CB600FE1EFE1CFE1BFE1AFE18FE17FE15FE1457
:102CC600FE13FE11FE10FE0FFE0DFE0CFE0BFE099E
:102CD600FE08FE06FE05FE04FE02FE01FE00FDFEE7
:102CE600FDFDFDFCFDFAFDF9FDF7FDF6FDF5FDF335
:102CF600FDF2FDF1FDEFFDEEFDEDFDEBFDEAFDE97B
:102D0600FDE7FDE6FDE5FDE3FDE2FDE1FDDFFDDEC0
:102D1600FDDDFDDBFDDAFDD9FDD7FDD6FDD5FDD305
:102D2600FDD2FDD1FDCFFDCEFDCDFDCCFDCAFDC949
:102D3600FDC8FDC6FDC5FDC4FDC2FDC1FDC0FDBE8D
:102D4600FDBDFDBCFDBBFDB9FDB8FDB7FDB5FDB4D0
:102D5600FDB3FDB2FDB0FDAFFDAEFDACFDABFDAA12
:102D6600FDA9FDA7FDA6FDA5FDA4FDA2FDA1FDA053
:102D7600FD9FFD9DFD9CFD9BFD99FD98FD97FD9694
:102D8600FD94FD93FD92FD91FD8FFD8EFD8DFD8CD5
:102D9600FD8AFD89FD88FD87FD86FD84FD83FD8214
:102DA600FD81FD7FFD7EFD7DFD7CFD7BFD79FD7852
:102DB600FD77FD76FD74FD73FD72FD71FD70FD6E90
:102DC600FD6DFD6CFD6BFD6AFD68FD67FD66FD65CD
:102DD600FD64FD62FD61FD60FD5FFD5EFD5DFD5B09
:102DE600FD5AFD59FD58FD57FD55FD54FD53FD5245
:102DF600FD51FD50FD4EFD4DFD4CFD4BFD4AFD497F
:102E0600FD48FD46FD45FD44FD43FD42FD41FD40B7
:102E1600FD3EFD3DFD3CFD3BFD3AFD39FD38FD36F1
:102E2600FD35FD34FD33FD32FD31FD30FD2FFD2E28
:102E3600FD2CFD2BFD2AFD29FD28FD27FD26FD2560
:102E4600FD24FD22FD21FD20FD1FFD1EFD1DFD1C97
:102E5600FD1BFD1AFD19FD18FD17FD15FD14FD13CB
:102E6600FD12FD11FD10FD0FFD0EFD0DFD0CFD0B00
:102E7600FD0AFD09FD08FD07FD06FD05FD03FD0232
:102E8600FD01FD00FCFFFCFEFCFDFCFCFCFBFCFA6E
:102E9600FCF9FCF8FCF7FCF6FCF5FCF4FCF3FCF2A0
:102EA600FCF1FCF0FCEFFCEEFCEDFCECFCEBFCEAD0
:102EB600FCE9FCE8FCE7FCE6FCE5FCE4FCE3FCE200
:102EC600FCE1FCE0FCDFFCDEFCDDFCDCFCDBFCDA30
:102ED600FCD9FCD8FCD7FCD6FCD5FCD4FCD3FCD35F
:102EE600FCD2FCD1FCD0FCCFFCCEFCCDFCCCFCCB88
:102EF600FCCAFCC9FCC8FCC7FCC6FCC5FCC4FCC4B7
:102F0600FCC3FCC2FCC1FCC0FCBFFCBEFCBDFCBCDF
:102F1600FCBBFCBAFCB9FCB9FCB8FCB7FCB6FCB50A
:102F2600FCB4FCB3FCB2FCB1FCB1FCB0FCAFFCAE33
:102F3600FCADFCACFCABFCAAFCAAFCA9FCA8FCA75B
:102F4600FCA6FCA5FCA4FCA4FCA3FCA2FCA1FCA082
:102F5600FC9FFC9FFC9EFC9DFC9CFC9BFC9AFC9AA7
:102F6600FC99FC98FC97FC96FC95FC95FC94FC93CC
:102F7600FC92FC91FC91FC90FC8FFC8EFC8DFC8DF0
:102F8600FC8CFC8BFC8AFC89FC89FC88FC87FC8613
:102F9600FC86FC85FC84FC83FC82FC82FC81FC8034
:102FA600FC7FFC7FFC7EFC7DFC7CFC7CFC7BFC7A55
:102FB600FC79FC79FC78FC77FC76FC76FC75FC7475
:102FC600FC74FC73FC72FC71FC71FC70FC6FFC6F92
:102FD600FC6EFC6DFC6CFC6CFC6BFC6AFC6AFC69B0
:102FE600FC68FC68FC67FC66FC66FC65FC64FC63CC
:102FF600FC63FC62FC61FC61FC60FC5FFC5FFC5EE8
:10300600FC5EFC5DFC5CFC5CFC5BFC5AFC5AFC59FF
:10301600FC58FC58FC57FC56FC56FC55FC55FC5419
:10302600FC53FC53FC52FC51FC51FC50FC50FC4F31
:10303600FC4EFC4EFC4DFC4DFC4CFC4BFC4BFC4A48
:10304600FC4AFC49FC49FC48FC47FC47FC46FC465C
:10305600FC45FC45FC44FC43FC43FC42FC42FC4171
:10306600FC41FC40FC40FC3FFC3EFC3EFC3DFC3D84
:10307600FC3CFC3CFC3BFC3BFC3AFC3AFC39FC3996
:10308600FC38FC38FC37FC37FC36FC36FC35FC35A6
:10309600FC34FC34FC33FC33FC32FC32FC31FC31B6
:1030A600FC30FC30FC2FFC2FFC2EFC2EFC2EFC2DC5
:1030B600FC2DFC2CFC2CFC2BFC2BFC2AFC2AFC29D2
:1030C600FC29FC29FC28FC28FC27FC27FC26FC26DE
:1030D600FC26FC25FC25FC24FC24FC24FC23FC23E8
:1030E600FC22FC22FC22FC21FC21FC20FC20FC20F2
:1030F600FC1FFC1FFC1EFC1EFC1EFC1DFC1DFC1DFB
:10310600FC1CFC1CFC1BFC1BFC1BFC1AFC1AFC1A02
:10311600FC19FC19FC19FC18FC18FC18FC17FC1708
:10312600FC17FC16FC16FC16FC15FC15FC15FC140D
:10313600FC14FC14FC14FC13FC13FC13FC12FC1210
:10314600FC12FC12FC11FC11FC11FC10FC10FC1012
:10315600FC10FC0FFC0FFC0FFC0FFC0EFC0EFC0E13
:10316600FC0EFC0DFC0DFC0DFC0DFC0CFC0CFC0C13
:10317600FC0CFC0BFC0BFC0BFC0BFC0AFC0AFC0A13
:10318600FC0AFC0AFC09FC09FC09FC09FC09FC0810
:10319600FC08FC08FC08FC08FC07FC07FC07FC070D
:1031A600FC07FC07FC06FC06FC06FC06FC06FC0607
:1031B600FC05FC05FC05FC05FC05FC05FC05FC0402
:1031C600FC04FC04FC04FC04FC04FC04FC04FC03FA
:1031D600FC03FC03FC03FC03FC03FC03FC03FC03F1
:1031E600FC02FC02FC02FC02FC02FC02FC02FC02E9
:1031F600FC02FC02FC02FC02FC01FC01FC01FC01DD
:10320600FC01FC01FC01FC01FC01FC01FC01FC01D0
:10321600FC01FC01FC01FC01FC01FC01FC01FC01C0
:10322600FC01FC01FC01FC01FC01FC01FC01FC01B0
:10323600FC01FC01FC01FC01FC01FC01FC01FC01A0
:10324600FC01FC01FC01FC01FC01FC01FC01FC0190
:10325600FC01FC01FC01FC01FC01FC01FC01FC0180
:10326600FC01FC01FC01FC01FC01FC02FC02FC026D
:10327600FC02FC02FC02FC02FC02FC02FC02FC0258
:10328600FC02FC03FC03FC03FC03FC03FC03FC0341
:10329600FC03FC03FC04FC04FC04FC04FC04FC042A
:1032A600FC04FC04FC05FC05FC05FC05FC05FC0512
:1032B600FC05FC06FC06FC06FC06FC06FC06FC07F8
:1032C600FC07FC07FC07FC07FC07FC08FC08FC08DD
:1032D600FC08FC08FC09FC09FC09FC09FC09FC0AC1
:1032E600FC0AFC0AFC0AFC0AFC0BFC0BFC0BFC0BA4
:1032F600FC0CFC0CFC0CFC0CFC0DFC0DFC0DFC0D84
:10330600FC0EFC0EFC0EFC0EFC0FFC0FFC0FFC0F63
:10331600FC10FC10FC10FC10FC11FC11FC11FC1242
:10332600FC12FC12FC12FC13FC13FC13FC14FC1420
:10333600FC14FC14FC15FC15FC15FC16FC16FC16FE
:10334600FC17FC17FC17FC18FC18FC18FC19FC19D8
:10335600FC19FC1AFC1AFC1AFC1BFC1BFC1BFC1CB3
:10336600FC1CFC1DFC1DFC1DFC1EFC1EFC1EFC1F8B
:10337600FC1FFC20FC20FC20FC21FC21FC22FC2262
:10338600FC22FC23FC23FC24FC24FC24FC25FC2539
:10339600FC26FC26FC26FC27FC27FC28FC28FC290E
:1033A600FC29FC29FC2AFC2AFC2BFC2BFC2CFC2CE3
:1033B600FC2DFC2DFC2EFC2EFC2EFC2FFC2FFC30B5
:1033C600FC30FC31FC31FC32FC32FC33FC33FC3487
:1033D600FC34FC35FC35FC36FC36FC37FC37FC3857
:1033E600FC38FC39FC39FC3AFC3AFC3BFC3BFC3C27
:1033F600FC3CFC3DFC3DFC3EFC3EFC3FFC40FC40F6
:10340600FC41FC41FC42FC42FC43FC43FC44FC45C1
:10341600FC45FC46FC46FC47FC47FC48FC49FC498D
:10342600FC4AFC4AFC4BFC4BFC4CFC4DFC4DFC4E58
:10343600FC4EFC4FFC50FC50FC51FC51FC52FC5322
:10344600FC53FC54FC55FC55FC56FC56FC57FC58EA
:10345600FC58FC59FC5AFC5AFC5BFC5CFC5CFC5DB1
:10346600FC5EFC5EFC5FFC5FFC60FC61FC61FC6278
:10347600FC63FC63FC64FC65FC66FC66FC67FC683C
:10348600FC68FC69FC6AFC6AFC6BFC6CFC6CFC6D01
:10349600FC6EFC6FFC6FFC70FC71FC71FC72FC73C3
:1034A600FC74FC74FC75FC76FC76FC77FC78FC7985
:1034B600FC79FC7AFC7BFC7CFC7CFC7DFC7EFC7F46
:1034C600FC7FFC80FC81FC82FC82FC83FC84FC8506
:1034D600FC86FC86FC87FC88FC89FC89FC8AFC8BC4
:1034E600FC8CFC8DFC8DFC8EFC8FFC90FC91FC9181
:1034F600FC92FC93FC94FC95FC95FC96FC97FC983E
:10350600FC99FC9AFC9AFC9BFC9CFC9DFC9EFC9FF7
:10351600FC9FFCA0FCA1FCA2FCA3FCA4FCA4FCA5B3
:10352600FCA6FCA7FCA8FCA9FCAAFCAAFCABFCAC6C
:10353600FCADFCAEFCAFFCB0FCB1FCB1FCB2FCB324
:10354600FCB4FCB5FCB6FCB7FCB8FCB9FCB9FCBADB
:10355600FCBBFCBCFCBDFCBEFCBFFCC0FCC1FCC291
:10356600FCC3FCC4FCC4FCC5FCC6FCC7FCC8FCC947
:10357600FCCAFCCBFCCCFCCDFCCEFCCFFCD0FCD1F9
:10358600FCD2FCD3FCD3FCD4FCD5FCD6FCD7FCD8AF
:10359600FCD9FCDAFCDBFCDCFCDDFCDEFCDFFCE061
:1035A600FCE1FCE2FCE3FCE4FCE5FCE6FCE7FCE811
:1035B600FCE9FCEAFCEBFCECFCEDFCEEFCEFFCF0C1
:1035C600FCF1FCF2FCF3FCF4FCF5FCF6FCF7FCF871
:1035D600FCF9FCFAFCFBFCFCFCFDFCFEFCFFFD0020
:1035E600FD01FD02FD03FD05FD06FD07FD08FD09C4
:1035F600FD0AFD0BFD0CFD0DFD0EFD0FFD10FD1171
:10360600FD12FD13FD14FD15FD17FD18FD19FD1A1C
:10361600FD1BFD1CFD1DFD1EFD1FFD20FD21FD22C8
:10362600FD24FD25FD26FD27FD28FD29FD2AFD2B70
:10363600FD2CFD2EFD2FFD30FD31FD32FD33FD3419
:10364600FD35FD36FD38FD39FD3AFD3BFD3CFD3DC2
:10365600FD3EFD40FD41FD42FD43FD44FD45FD4669
:10366600FD48FD49FD4AFD4BFD4CFD4DFD4FFD500E
:10367600FD51FD52FD53FD54FD55FD57FD58FD59B5
:10368600FD5AFD5BFD5DFD5EFD5FFD60FD61FD625A
:10369600FD64FD65FD66FD67FD68FD6AFD6BFD6CFD
:1036A600FD6DFD6EFD70FD71FD72FD73FD74FD76A1
:1036B600FD77FD78FD79FD7BFD7CFD7DFD7EFD7F43
:1036C600FD81FD82FD83FD84FD86FD87FD88FD89E4
:1036D600FD8BFD8CFD8DFD8EFD8FFD91FD92FD9385
:1036E600FD94FD96FD97FD98FD99FD9BFD9CFD9D26
:1036F600FD9FFDA0FDA1FDA2FDA4FDA5FDA6FDA7C4
:10370600FDA9FDAAFDABFDACFDAEFDAFFDB0FDB262
:10371600FDB3FDB4FDB5FDB7FDB8FDB9FDBBFDBC00
:10372600FDBDFDBEFDC0FDC1FDC2FDC4FDC5FDC69E
:10373600FDC8FDC9FDCAFDCCFDCDFDCEFDCFFDD139
:10374600FDD2FDD3FDD5FDD6FDD7FDD9FDDAFDDBD6
:10375600FDDDFDDEFDDFFDE1FDE2FDE3FDE5FDE670
:10376600FDE7FDE9FDEAFDEBFDEDFDEEFDEFFDF10B
:10377600FDF2FDF3FDF5FDF6FDF7FDF9FDFAFDFCA5
:10378600FDFDFDFEFE00FE01FE02FE04FE05FE0638
:10379600FE08FE09FE0BFE0CFE0DFE0FFE10FE11CE
:1037A600FE13FE14FE16FE17FE18FE1AFE1BFE1C66
:1037B600FE1EFE1FFE21FE22FE23FE25FE26FE28FD
:1037C600FE29FE2AFE2CFE2DFE2FFE30FE31FE3394
:1037D600FE34FE36FE37FE38FE3AFE3BFE3DFE3E2A
:1037E600FE3FFE41FE42FE44FE45FE46FE48FE49C1
:1037F600FE4BFE4CFE4EFE4FFE50FE52FE53FE5555
:10380600FE56FE58FE59FE5AFE5CFE5DFE5FFE60E9
:10381600FE62FE63FE64FE66FE67FE69FE6AFE6C7D
:10382600FE6DFE6FFE70FE71FE73FE74FE76FE7711
:10383600FE79FE7AFE7CFE7DFE7EFE80FE81FE83A4
:10384600FE84FE86FE87FE89FE8AFE8CFE8DFE8F36
:10385600FE90FE91FE93FE94FE96FE97FE99FE9ACA
:10386600FE9CFE9DFE9FFEA0FEA2FEA3FEA5FEA65A
:10387600FEA8FEA9FEAAFEACFEADFEAFFEB0FEB2ED
:10388600FEB3FEB5FEB6FEB8FEB9FEBBFEBCFEBE7E
:10389600FEBFFEC1FEC2FEC4FEC5FEC7FEC8FECA0E
:1038A600FECBFECDFECEFED0FED1FED3FED4FED69E
:1038B600FED7FED9FEDAFEDCFEDDFEDFFEE0FEE22E
:1038C600FEE3FEE5FEE6FEE8FEE9FEEBFEECFEEEBE
:1038D600FEEFFEF1FEF2FEF4FEF5FEF7FEF8FEFA4E
:1038E600FEFCFEFDFEFFFF00FF02FF03FF05FF06D5
:1038F600FF08FF09FF0BFF0CFF0EFF0FFF11FF1262
:10390600FF14FF15FF17FF18FF1AFF1CFF1DFF1FEF
:10391600FF20FF22FF23FF25FF26FF28FF29FF2B7D
:10392600FF2CFF2EFF2FFF31FF33FF34FF36FF370B
:10393600FF39FF3AFF3CFF3DFF3FFF40FF42FF4498
:10394600FF45FF47FF48FF4AFF4BFF4DFF4EFF5025
:10395600FF51FF53FF55FF56FF58FF59FF5BFF5CB2
:10396600FF5EFF5FFF61FF62FF64FF66FF67FF693F
:10397600FF6AFF6CFF6DFF6FFF70FF72FF74FF75CC
:10398600FF77FF78FF7AFF7BFF7DFF7EFF80FF8258
:10399600FF83FF85FF86FF88FF89FF8BFF8DFF8EE4
:1039A600FF90FF91FF93FF94FF96FF97FF99FF9B70
:1039B600FF9CFF9EFF9FFFA1FFA2FFA4FFA6FFA7FC
:1039C600FFA9FFAAFFACFFADFFAFFFB0FFB2FFB488
:1039D600FFB5FFB7FFB8FFBAFFBBFFBDFFBFFFC014
:1039E600FFC2FFC3FFC5FFC6FFC8FFCAFFCBFFCD9F
:1039F600FFCEFFD0FFD1FFD3FFD5FFD6FFD8FFD92B
:103A0600FFDBFFDCFFDEFFE0FFE1FFE3FFE4FFE6B5
:103A1600FFE7FFE9FFEBFFECFFEEFFEFFFF1FFF241
:103A2600FFF4FFF6FFF7FFF9FFFAFFFCFFFDFFFFCC
:03000000020C00EF
:03000300021A03DB
:03000B00021A06D0
:03001300021A09C5
:03001B00021A0CBA
:03002300021A0FAF
:03002B00021A12A4
:03003300021A1599
:03003B00021A188E
:03004300021A1B83
:03004B00021A1E78
:03005300021A216D
:03005B00021A2462
:03006300021A2757
:03006B00021A2A4C
:03007300021A2D41
:03007B00021A3036
:03008300021A332B
:03008B00021A3620
:03009300021A3915
:03009B00021A3C0A
:0300A300021A3FFF
:100C0000787FE4F6D8FD9000007F007E20E4F0A31A
:0A0C1000DFFCDEFA758162020C556C
:100C1A00021389E493A3F8E493A34003F68001F254
:100C2A0008DFF48029E493A3F85407240CC8C333DB
:100C3A00C4540F4420C8834004F456800146F6DFAA
:100C4A00E4800B0102040810204080904FEAE47E01
:100C5A00019360BCA3FF543F30E509541FFEE4939F
:100C6A00A360010ECF54C025E060A840B8E493A366
:100C7A00FAE493A3F8E493A3C8C582C8CAC583CA91
:100C8A00F0A3C8C582C8CAC583CADFE9DEE780BE49
:0150A9000006
:100C9A00E709F608DFFA8046E709F208DFFA803E3C
:100CAA0088828C83E709F0A3DFFA8032E309F60829
:100CBA00DFFA8078E309F208DFFA807088828C8391
:100CCA00E309F0A3DFFA806489828A83E0A3F60845
:100CDA00DFFA805889828A83E0A3F208DFFA804C1F
:100CEA0080D280FA80C680D4806980F280338010F6
:100CFA0080A680EA809A80A880DA80E280CA80335F
:100D0A0089828A83ECFAE493A3C8C582C8CCC583D6
:100D1A00CCF0A3C8C582C8CCC583CCDFE9DEE780A6
:100D2A000D89828A83E493A3F608DFF9ECFAA9F025
:100D3A00EDFB2289828A83ECFAE0A3C8C582C8CC7B
:100D4A00C583CCF0A3C8C582C8CCC583CCDFEADE94
:100D5A00E880DB89828A83E493A3F208DFF980CCF6
:100D6A0088F0EF60010E4E60C388F0ED2402B404EF
:100D7A000050B9F582EB2402B4040050AF23234596
:060D8A008223900CEA73C5
:100D9000BB010689828A83E0225002E722BBFE0261
:090DA000E32289828A83E4932294
:100DA900BB010CE58229F582E5833AF583E02250FF
:100DB90006E92582F8E622BBFE06E92582F8E22249
:0D0DC900E58229F582E5833AF583E4932263
:100DD600BB010689828A83F0225002F722BBFE01FC
:020DE600F322F6
:100DE800EF8DF0A4A8F0CF8CF0A428CE8DF0A42E1F
:020DF800FE22D9
:100DFA00BC000BBE0029EF8DF084FFADF022E4CCDD
:100E0A00F875F008EF2FFFEE33FEEC33FCEE9DECA5
:100E1A00984005FCEE9DFE0FD5F0E9E4CEFD22EDEB
:100E2A00F8F5F0EE8420D21CFEADF075F008EF2F35
:100E3A00FFED33FD4007985006D5F0F222C398FD26
:050E4A000FD5F0EA22C3
:100E4F00C5F0F8A3E028F0C5F0F8E582158270022E
:060E5F001583E038F022CB
:100E6500A3F8E0C5F025F0F0E58215827002158340
:060E7500E0C838F0E8229D
:100E7B00E88FF0A4CC8BF0A42CFCE98EF0A42CFC16
:100E8B008AF0EDA42CFCEA8EF0A4CDA8F08BF0A494
:100E9B002DCC3825F0FDE98FF0A42CCD35F0FCEBF3
:100EAB008EF0A4FEA9F0EB8FF0A4CFC5F02ECD39B8
:0F0EBB00FEE43CFCEAA42DCE35F0FDE43CFC2225
:100ECA0075F008758200EF2FFFEE33FECD33CDCCDF
:100EDA0033CCC58233C5829BED9AEC99E582984062
:100EEA000CF582EE9BFEED9AFDEC99FC0FD5F0D63F
:100EFA00E4CEFBE4CDFAE4CCF9A88222B800C1B969
:100F0A000059BA002DEC8BF084CFCECDFCE5F0CBA6
:100F1A00F97818EF2FFFEE33FEED33FDEC33FCEBDF
:100F2A0033FB10D703994004EB99FB0FD8E5E4F99A
:100F3A00FA227818EF2FFFEE33FEED33FDEC33FC87
:100F4A00C933C910D7059BE99A4007EC9BFCE99A7B
:100F5A00F90FD8E0E4C9FAE4CCFB2275F010EF2FC0
:100F6A00FFEE33FEED33FDCC33CCC833C810D707C0
:100F7A009BEC9AE899400AED9BFDEC9AFCE899F8FB
:0E0F8A000FD5F0DAE4CDFBE4CCFAE4C8F9228E
:105C6F00C2D5E830E70FB2D5E4C39BFBE49AFAE460
:105C7F0099F9E498F8EC30E717B2D5125CA5120F3A
:105C8F0006E4C39BFBE49AFAE499F9E498F88003DD
:105C9F00120F0630D50DE4C39FFFE49EFEE49DFD79
:045CAF00E49CFC2253
:100F9800EB9FF5F0EA9E42F0E99D42F0EC6480C8D0
:060FA80064809845F02270
:100FAE00EB9FF5F0EA9E42F0E99D42F0E89C45F099
:010FBE002210
:100FBF00E8600FECC313FCED13FDEE13FEEF13FF10
:030FCF00D8F12234
:100FD200E8600FEFC333FFEE33FEED33FDEC33FC7D
:030FE200D8F12221
:100FE5007401FF3395E0FEFDFCA3A3A3E0CF2FF032
:100FF500E582158270021583E0CE3EF0E58215820A
:1010050070021583E0CD3DF0E582158270021583EF
:05101500E0CC3CF022DC
:0C101A00ECF0A3EDF0A3EEF0A3EFF02249
:10102600A8828583F0D083D08212103D12103D1223
:10103600103D12103DE473E493A3C583C5F0C58348
:10104600C8C582C8F0A3C583C5F0C583C8C582C814
:011056002277
:0C105700A42582F582E5F03583F58322A4
:10106300D083D082F8E4937012740193700DA3A31C
:1010730093F8740193F5828883E473740293686030
:06108300EFA3A3A380DF30
:00000001FF
